:020000040000FA
:020000001928BD
:08000800F9280D340A345234CA
:1000100061346E3467346534723420345634653458
:1000200072342E34203430342E3433340D340A34C8
:100030000034DE20622127210A304F21831203136E
:100040000430A000A10105304321901010140530A8
:100050009700F4010D302F210A302F213A302F2143
:100060008F018E01741C322874107508643C0319CA
:100070004A287508663C0319AB287508623C0319C9
:1000800095287508673C031971287508683C0319A1
:100090006428322883120313741C4C2874107508CA
:1000A0001B3C03192A2830307502F600093C031C5A
:1000B0002A280430A000F60AF60B61282008BF2089
:1000C0002A280430A0075C288312031305182A2865
:1000D0006A206428831203139C20880020084F2183
:1000E0000800831203138F018E01871483160313F4
:1000F0000C14831203130714F4188D28741C7C2825
:10010000741075081B3C031D7C288710071083168C
:1001100003130C10831203132A28F4102208BF20A3
:100120002308BF20871007102A28831203139C205E
:10013000880020084F212A2883120313A1030730C7
:10014000A10521088207083404340234013408343C
:1001500004340234013483120313B02088002A28A7
:1001600083120313A10A0730A1052108820708346E
:100170000434023401340834043402340134831268
:100180000313F700F039F8000310F80C0310F80C13
:100190000310F80C0310F80C0A3078023030031802
:1001A000373078072F210F307705F8000A307802B2
:1001B00030300318373078072F21080083120313DB
:1001C000871009108910831603130B308500073040
:1001D0009F00FF308600E4308700F0308800043054
:1001E00089008312031387100710091089108801F2
:1001F0000800F200030E8301F3008C1E0529722112
:10020000F5008C1274142F2162210C1D1129871006
:1002100007101608A2001508A300F4140C118F0192
:100220008E010C1C2229871007100C108316031353
:100230000C1083120313FF30A200FF30A300F4144C
:100240008F018E01730E8300F20E720E0900831669
:1002500003130C150B178B17831203130800831657
:100260000313981C3129F0000C309900181518124E
:1002700083120313981783160313981670088312BA
:10028000031399000800F1004D21F0007008031DD0
:100290004A2908002F21F10A44297108820083129B
:1002A0000313F9005821F90B522983120313080094
:1002B00083120313E530FA000000FA0B5C29831265
:1002C00003130800831603130C3099001815181235
:1002D0008312031398171816831603138C168312B0
:0A02E000031308001A0818120800A2
:02400E00313D42
:00000001FF
